:1000000044C05CC05BC05AC059C058C057C056C03D
:1000100055C054C053C052C051C050C04FC04EC054
:100020004DC04CC04BC057524F4E470A004F4B215A
:1000300020596F7527726520696E2E205A686520D9
:100040005A656B7269742057657572642049733AFA
:100050000A00456E7465722074686520342D6469E9
:1000600067697420636F64652E0A00526561647964
:100070002E0A0045464765666700202B2D2E30313D
:100080003233343536373839680011241FBECFED8E
:10009000CDBF10E0A0E6B0E0E0E6F6E002C00590DB
:1000A0000D92A637B107D9F710E0A6E7B0E001C07E
:1000B0001D92AC37B107E1F706D0D0C2A1CF5F9B4C
:1000C000FECF8CB108952F923F924F925F926F9224
:1000D0007F928F929F92AF92BF92CF92DF92EF92D8
:1000E000FF920F931F93DF93CF9300D000D000D0E7
:1000F000CDB7DEB783E390E099D000D08BE690E0F7
:10010000EDB7FEB79283818320D20F900F9052E516
:10011000252E50E0352E2E010894411C511C45E03F
:10012000642E712C6C0E7D1E30EDE32E37E0F32E25
:1001300026E2822E20E0922E9DE2A92E90E0B92E9A
:100140008BEBC82E8FEFD82E00D0EDB7FEB73282E2
:100150002182FBD1F2010F900F905F9BFECF8CB1FB
:10016000865F8193E615F705C1F78981803419F020
:1001700020E030E005C0C7010197F1F721E030E051
:100180008A818D3319F020E030E006C02115310559
:1001900019F0C7010197F1F78B81823419F020E043
:1001A00030E006C02115310519F0C7010197F1F7BC
:1001B0008C818C3329F5232B19F1C7010197F1F7B5
:1001C00000D0EDB7FEB7B282A182BFD100E010E04F
:1001D0000F900F90C601801B910BF801E05AFF4F62
:1001E0002081332727FD3095820F931FD1D10F5FD8
:1001F0001F4F0730110571F78AE090E0C9D1A4CFF5
:1002000000D0EDB7FEB7928281829FD10F900F9000
:100210009BCF1F93182F8A3011F48DE0FADF5D9B7E
:10022000FECF1CB980E090E01F91089528E12AB923
:1002300089B9892F990F990B82B988E690E090933C
:100240007900809378000895ABE0B0E0E9E2F1E056
:1002500012C15C014B017A01FC0117821682838175
:1002600081FD08C06FEF7FEFFEC042E050E0E40E7A
:10027000F51E04C03E010894611C711CF501D38079
:10028000F401D3FC8591D3FE81914F01882309F4B9
:10029000E7C0853259F4D3FC6591D3FE61914F01DB
:1002A000653219F0062F10E01AC085E290E029C0EF
:1002B000002309F4D5C08AE790E0602F70E00ED1EA
:1002C000892B39F4033211F4106103C00C3661F448
:1002D0001068F401D3FC0591D3FE01914F0117FF83
:1002E000E7CF002309F4BCC083E790E0602F70E003
:1002F000F5D0892B49F044E050E0E40EF51E8FE381
:1003000090E0B501F6D0BACF033629F0033771F08B
:100310000335E1F40AC087010E5F1F4FF7018081AA
:100320009181B501E6D07801A9CF1160F701C080B5
:10033000D18003C090E0B501DCD0F60110FD8591BD
:1003400010FF81916F018823A9F78FCF043611F038
:10035000093639F517FF08C0F70120813181428144
:10036000538184E090E00AC0F701808191819C0173
:10037000442737FD4095542F82E090E0E80EF91EA7
:100380001F7E57FF08C050954095309521953F4FEF
:100390004F4F5F4F1064CA01B901A3012AE030E05A
:1003A00034C00037A9F0013730F40835B1F00F360A
:1003B00009F056C006C0053739F0083709F050C0BB
:1003C00008C028E030E00CC01F7E2AE030E008C002
:1003D0001061146220E130E003C0146020E132E0DB
:1003E00017FF08C0F701608171818281938144E029
:1003F00050E008C0F70180819181BC0180E090E06D
:1004000042E050E0E40EF51EA301C8D0D82ED61865
:10041000012F10E006FF04C08DE290E0B50169D025
:1004200004FF13C0FE01ED0DF11D8081803369F0E2
:1004300080E390E0B5015DD002FF07C0007210704C
:10044000C801885A9F4FB50154D0DA94F301ED0DDD
:10045000F11D808190E0B5014CD0DD20B1F70ECFC9
:10046000F50166817781CB012B96EEE020C02F92BB
:100470003F924F925F926F927F928F929F92AF9234
:10048000BF92CF92DF92EF92FF920F931F93CF9381
:10049000DF93CDB7DEB7CA1BDB0B0FB6F894DEBF18
:1004A0000FBECDBF09942A88398848885F846E843E
:1004B0007D848C849B84AA84B984C884DF80EE8088
:1004C000FD800C811B81AA81B981CE0FD11D0FB691
:1004D000F894DEBF0FBECDBFED010895FC0105907D
:1004E000061621F00020D9F7C00108953197CF01F9
:1004F00008950F931F93CF93DF938C01EB018B81B2
:1005000081FF1BC082FF0DC02E813F818C819D81A8
:100510002817390764F4E881F9810193F983E883A6
:1005200006C0E885F985802F0995892B31F48E81E5
:100530009F8101969F838E8302C00FEF1FEFC8013A
:10054000DF91CF911F910F910895A0E0B0E0EAEA0A
:10055000F2E09DCFFE01359661917191A0917800F6
:10056000B091790013968C911397886013968C93B1
:100570008091780090917900AF0166DEE09178007B
:10058000F09179002381277F23832096E2E09BCF9F
:100590006091780070917900ACDF0895FA01AA2784
:1005A000283061F1203191F1E8946F936E7F6E5F96
:1005B0007F4F8F4F9F4FAF4FB1E040D0B4E03ED060
:1005C000670F781F891F9A1FA11D680F791F8A1F47
:1005D000911DA11D6A0F711D811D911DA11D22D0AC
:1005E00009F468943F91062E000C3019000C000CA1
:1005F0003019305D3193CEF6CF010895462F477004
:10060000405D4193B3E00FD0C9F7F6CF462F4F704E
:10061000405D4A3318F0495D31FD4052419302D0AC
:10062000A9F7EACFB4E0A695979587957795679552
:10063000BA95C9F700976105710508959B01AC0152
:100640000A2E06945795479537952795BA95C9F779
:10065000620F731F841F951FA01D0895F894FFCF8C
:10066000B7B5BAADABBFAF0000000002000000009C
:060670000901000000007A
:00000001FF
